:1000000000000A128A110E28FE00030EF0000408F8
:10001000F1000A08F2000A168A1137288301030842
:08002000A0000A128A11C52F8D
:10002A00403083129F00803083169F0008006400CE
:10003A008001840A04060319003404061D28D230FC
:10004A00CD009930CE000A128A15CF270A128A11DA
:10005A00A0300A128A15CB270A128A11A0300A1276
:10006A008A156B270A128A112408D0002308CF00A8
:10007A0050040319782804305002453003194F02FE
:10008A000318782850088316EE0083124F08831647
:10009A00ED0004308312A100A20183166E088312B8
:1000AA00A40083166D088312A3000A128A15282455
:1000BA000A128A11CC3083120313C0009A30C1008D
:1000CA0083166E088312C30083166D088312C2005A
:1000DA00A0300A128A155727A030CD000130CE0071
:1000EA000A128A15462F6A30CD009A30CE000A12BB
:1000FA008A15462F031003178312201E031400309B
:10010A000318013083160313EF00640017308312BB
:10011A0003178500F830831603138100073003178D
:10012A0088000313850086010317890103138701D9
:10013A008312870186018501861285126430CF00F9
:10014A00D0010A128A1528210A128A118B130A165B
:10015A008A1150270A128A110A128A11B5270A121D
:10016A008A110A168A11B0260A128A110A128A11EB
:10017A0015200A128A118B17F401F40AF5010A12E2
:10018A008A1550240A128A11750883160313CE00A1
:10019A007408CD0003300A128A155C240A128A11E7
:1001AA0083160313DA0063308312C0009930C1004A
:1001BA006A30C2009A30C300A0300A128A15572743
:1001CA000A128A11A030CD000130CE000A128A1517
:1001DA0046270A128A1183165A08031937299130B9
:1001EA008312CD009930CE000A128A1546270A12C8
:1001FA008A110430F400F5010A128A1550240A12F1
:10020A008A11750883160313EE007408ED00063090
:10021A00F400F5010A128A1550240A128A11750887
:10022A0083160313D8007408D7001030F400F501C0
:10023A000A128A1550240A128A11750883160313A2
:10024A00E0007408DF001E300A128A1580240A12A0
:10025A008A11003A031D372900300A128A15AA2387
:10026A000A128A1183120317D730A201A3010313BA
:10027A00CD009A30CE000A128A15CF270A128A11A7
:10028A000A128A15DC270A128A11031C79290A1212
:10029A008A1174270A128A1183120317A300083AD3
:1002AA00031D6A29220803197929A2032308F300E6
:1002BA000A128A1157270A128A112030F3000A12E9
:1002CA008A1157270A128A1170292208A03E84002F
:1002DA0023088000A20A831203172308F3000A12D4
:1002EA008A1157270A128A116400831603135708C2
:1002FA0058040319B5290A168A1103200A128A1109
:10030A0073088312ED007408EE0083165808F4008F
:10031A005708F3003C30F500F6010A168A118E26BA
:10032A000A128A1174086E02031D9D2973086D0250
:10033A00031CB529C430CD009A30CE000A128A15A2
:10034A0046270A128A110A168A1154230A128A1196
:10035A0005308316EF0083120317A201A20ABF29F0
:10036A000D308312031723060319BF291F302202F7
:10037A00031C452922089F3E8400A0308317800170
:10038A000A128A156B270A128A1124080317A10078
:10039A00031323080317A00021080313EC00031713
:1003AA0020080313EB000A128A15AB240A128A11D9
:1003BA003729A000F8110C18F815831603130C102E
:1003CA0083125F088316A100A20183125E088316B6
:1003DA00A300A40183125D088316A500A601831257
:1003EA005C088316A700A80183125B08FF3E8316E8
:1003FA00A900FF3003180030AA002008643EAB00B1
:10040A00003003180130AC00831260088316B10073
:10041A00A130B2012B220A128A114F088316C80092
:10042A0083124E088316C70083124D088316C6002E
:10043A0083124C088316C500F81D272A8316031356
:10044A000C140800831603130C1008008312DA0038
:10045A000A3E84000D240A128A11031D362A4630E8
:10046A005002031C462A831203135A080A3E8400C8
:10047A000D240A128A11031D442A8B305002031CD0
:10048A004E2AFF3083120313D600D700D800D900B2
:10049A00C12A831203135A08083E840083130008F2
:1004AA00BE00840A0008BF00BE0A0319BF0A5A0820
:1004BA000A3E84000008BC00840A0008BD006C30B3
:1004CA00BC070318BD0A0730BD075A08063E840058
:1004DA000008C000840A0008C100CA220A128A1150
:1004EA003F08D9003E08D8003D08D7003C08D6008E
:1004FA00B230BC000730BD00BE01BE0ABF01C00158
:10050A00C00AC101CA220A128A113C08D6023D0851
:10051A00031C3D0FD7023E08031C3E0FD8023F08BA
:10052A00031C3F0FD9025A08043EF4231830A500D1
:10053A00A601A701A8010A168A1121230A128A1103
:10054A0018240A128A115A08023EF4230A128A113E
:10055A002F240A168A1121230A128A1118240A1230
:10056A008A115A08F4230A128A112F240A168A11A8
:10057A0021230A128A1118245908CF005808CE00DC
:10058A005708CD005608CC0008003F08AB003E08CB
:10059A00AA005B230A128A1140082A07C8004108E8
:1005AA000318410A2B07C9000030CA01CB013F02D8
:1005BA00033003193E02031C0A2B3D08AF003C0816
:1005CA00AE0032230A128A112E082F04031DF02AC4
:1005DA000230C600F22AC601C60AC7014608C2008E
:1005EA004708C3000030C31BFF30C400C5004208DF
:1005FA00C8024308031C430FC9024408031C440FE2
:10060A00CA024508031C450FCB020130BC02003068
:10061A00031CBD03BD023D08AB003C08AA007B23B6
:10062A002A08C8072B0803110318013E031DC9072E
:10063A002C0803110318013E031DCA072D080311D4
:10064A000318013E031DCB074B08BF004A08BE0032
:10065A004908BD004808BC0008009030B001B00A43
:10066A00AA000130AB002F08AD002E08AC000A1614
:10067A008A116A260A128A112A082B040319572B8F
:10068A002E080339031D562B6430AA00AB012F082C
:10069A00AD002E08AC000A168A116A262A082B0415
:1006AA000319B0013008AE00AF0108006430A3009E
:1006BA00A4012B08F4002A08F300F130F5000B30EE
:1006CA00F6000A168A118E260A128A117308413E0A
:1006DA00A50074080318013EF43EA6000A168A1102
:1006EA0040262408AB002308AA0008006430A300AF
:1006FA00A4012B08A6002A08A5000A168A1140267A
:10070A000A128A112308AE002408AF009030B00103
:10071A00B101A3000130A4002B08A6002A08A500F5
:10072A000A168A1140260A128A112308B2002408DE
:10073A00B300B401B5012B08B7002A08B6000310AC
:10074A00B70CB60C0310B70CB60C3608B80037084D
:10075A00B900BA01BB012A08A1002B08A200013086
:10076A00A301A401A801A701A6006D30A5000A16DD
:10077A008A1121230A128A112108B80722080318AC
:10078A00220FB90723080318230FBA0724080318EE
:10079A00240ABB073808B20739080318390FB30708
:1007AA003A0803183A0FB4073B0803183B0AB5077F
:1007BA002E08B2022F08031C2F0FB3023008031CA5
:1007CA00300FB4023108031C310FB5023508AD00F1
:1007DA003408AC003308AB003208AA0008008400D1
:1007EA0083130008D000840A0008D1005008D20000
:1007FA005108D3000030D31BFF30D400D50059086C
:10080A00A4005808A3005708A2005608A10008002F
:10081A0083130008D000840A0008D100803AFF0040
:10082A0080307F0208002108D20722080318220F0D
:10083A00D30723080318230FD40724080318240A0C
:10084A00D5075508D9005408D8005308D7005208CC
:10085A00D60008003C30A500A601A701A80108009F
:10086A0001308316031788000313850083120615C7
:10087A006430CF00D0010A128A1528210A128A117F
:10088A0000300A128A15C3210A128A117408E1007B
:10089A007308E00006116108A5006008A400AC24F2
:1008AA000A128A112408B9002508BA002608BB00D2
:1008BA0083164E088312A50083164D088312A400DE
:1008CA00AC240A128A112408AA002508AB002608BB
:1008DA00AC007A30A701A8004430A90019260A12F0
:1008EA008A112708B6002808B7002908B800812607
:1008FA000A128A113608C5003708C6003808C70028
:10090A00BC240A128A114608E3004508E20063087B
:10091A00A5006208A400AC240A128A112408D50092
:10092A002508D6002608D7003F30D201D301D400CB
:10093A0017250A128A115208C5005308C60054081E
:10094A00C700BC244608DF004508DE00080024086A
:10095A00F3002508F4008E30F501F600F701D725DB
:10096A007308A4007408A5007508A6000800F926F3
:10097A000A128A1103104A0D4B0DD1005108031DAA
:10098A00CB2CC501C601C701C8010800F9260A1205
:10099A008A1117300310CB0CCA0CC90CFF3E031D79
:1009AA00CF2C4908CC00C617C7014508CD00460818
:1009BA00CE004708CF008E30D001D102D11FF22CD1
:1009CA005108803A8F3E031CC62C0310D00CCF0C62
:1009DA00CE0CCD0CD10FEA2C002D18305102031881
:1009EA00C62C51080319002D0310CD0DCE0DCF0DC5
:1009FA00D00DD103F62C4C0803190E2DCD09CE09C2
:100A0A00CF09D009CD0A0319CE0A0319CF0A03194F
:100A1A00D00A5008C8004F08C7004E08C6004D0843
:100A2A00C50008005208D8005308D9005408DA0053
:100A3A000310590D5A0DDD005508D8005608D90083
:100A4A005708DA000310590D5A0DDC005D08031926
:100A5A003A2D5C085D025C080318422DD8005D0837
:100A6A00D80219305802031C412D5508D2005608E5
:100A7A00D3005708D40008005C08031908005D0871
:100A8A005C020318502D5D08D8005C08D8021930A2
:100A9A005802031808000630DB00D41BDB17D71BEB
:100AAA005B17D317D401D617D7015C085D02031868
:100ABA00772D0310D50DD60DD70DDC035C085D0626
:100ACA000319722DDB035B0807390319722D5E2D9A
:100ADA000310D40CD30CD20CDD0A5D085C06031992
:100AEA00932D6D2D5D085C020318932D0310D20D12
:100AFA00D30DD40DDD035C085D0603198F2DDB03CE
:100B0A005B08073903198F2D7B2D0310D70CD60CE0
:100B1A00D50CDC0A5D085C06031D8A2DDB1F9E2DA1
:100B2A00FF30D206D306D406D20A0319D30A031910
:100B3A00D40A5B1FA92DFF30D506D606D706D50ADB
:100B4A000319D60A0319D70ADB015208D507530835
:100B5A0003110318530A031DD60754080311031877
:100B6A00540A031DD707D71FC52DFF30D506D60651
:100B7A00D706D50A0319D60A0319D70ADB01DB0AF5
:100B8A005508F3005608F4005708F5005D08F6000A
:100B9A005B08F700D7257308D2007408D3007508DC
:100BAA00D400080076080319DF2D7508740473044D
:100BBA00031DE82DF301F401F5010800F60A0310FC
:100BCA00F50CF40CF30CFE3075050319F72DE32D23
:100BDA00F60AF30A0319F40A0319F50A0310F50CC5
:100BEA00F40CF30CFF3075050319052EED2D0230B8
:100BFA007602031C072EF6030310F30DF40DF50D10
:100C0A00F41FFC2D761CF4130310F60C7608A300CF
:100C1A00A201A1012108F3042208F4042308F5041F
:100C2A007708031DF51708002A08AD002B08AE0047
:100C3A002C08AF0003102E0D2F0DB4003408031D2D
:100C4A002A2EA701A801A90108002708AD00280833
:100C5A00AE002908AF0003102E0D2F0DB500350880
:100C6A00031D3B2EA701A801A90108008930B10183
:100C7A00B201B3013507AD00B4022C08B50029084A
:100C8A00B5068030B5051830AB17AC01A817A90115
:100C9A00B0000310B10DB20DB30D29082C02031DCB
:100CAA005C2E28082B02031D5C2E27082A02031C2F
:100CBA006A2E2708AA022808031C280FAB02290853
:100CCA00031C290AAC0231140310AA0DAB0DAC0D9A
:100CDA00B00B4E2E3108F3003208F4003308F50049
:100CEA003408F6003508F700D7257308A7007408FA
:100CFA00A8007508A90008003608BC003708BD001E
:100D0A003808BE0003103D0D3E0DBF003F08031D0D
:100D1A00922EB601B701B80108003908BC003A089A
:100D2A00BD003B08BE0003103D0D3E0DC400440843
:100D3A00031DA32EB601B701B801080044087B3E83
:100D4A00BF073808C4003B08C4068030C405073012
:100D5A00B717BA17BB01C001C101C201C300361CD3
:100D6A00BD2EEE260A128A1103183B0A031DC2077A
:100D7A000310B80CB70CB60C0310B90DBA0DBB0DA5
:100D8A00C30BB42E0930C300361CD22EEE260A122B
:100D9A008A1103183B0A031DC2070310B80CB70CCB
:100DAA00B60C0310C20CC10CC00CC30BC92E4008F0
:100DBA00F3004108F4004208F5003F08F600440831
:100DCA00F700D7257308B6007408B7007508B8008D
:100DDA0008003908C0073A08031103183A0A031D24
:100DEA00C1073B08031108004508C9004608CA00A4
:100DFA004708CB000800FF0007308A007F088207F7
:100E0A00052F0A128A11572FA300A4003D2F230889
:100E1A00240603193D2F2030F30057270A128A119E
:100E2A000830F30057270A128A118312A4033D2FB0
:100E3A000830F30057270A128A112030F300572787
:100E4A000A128A110830F30057270A128A118312EC
:100E5A00A4032408230203183D2F1D2F240884000D
:100E6A008001230808002408840021088000A40ABD
:100E7A006C270A128A118312A100A2012208003AE1
:100E8A000319482F382F2108083A03190C2F023A60
:100E9A000319332F073A0319332F183A03192E2F40
:100EAA00382F0800831603135D08013E0F395E06CA
:100EBA000319572F8B135D08103E8400730883179C
:100ECA008000DD0A0F30DD050C168B170800742729
:100EDA000A128A11F400F3005727740808000A124C
:100EEA008A15DC270A128A1103187D2F6400742FD1
:100EFA008B1383165B08903E840083170008F30067
:100F0A00DB0A0F30DB058B1773080800D4004C3A54
:100F1A00031D912F0516922F85153230CF00D0016F
:100F2A000A128A1528210A128A114C3083120313D5
:100F3A005406031DA22F0512A32F8511AB30C00042
:100F4A009A30C1005408C200A030C3010A128A159F
:100F5A005727A030CD000130CE000A128A15462F3D
:100F6A000F3083129000101080308F0000308E01F5
:0A0F7A00101483160C140B17080066
:100F8A00C530F801F901FA0183138400E1300A122D
:100F9A008A111C200A128A11903083178400ED30BE
:100FAA000A128A111C200A128A1110308400203079
:100FBA000A128A111C2083169F30E1009A30E2003F
:100FCA009930E3009A30E400B530E5009A30E60043
:100FDA00B030E7009A30E800D630E9009A30EA00EB
:100FEA00DA30EB009A30EC003C30ED00EE01830180
:060FFA000A128A117F2893
:101010008312031306160530CF00D00128210A12CF
:101020008A15831203138615EA30F901CD00993031
:10103000CE0046270A128A15D401D5010030550288
:101040001E3003195402031835286400E830831257
:101050000313CF000330D00028210A128A1583120F
:101060000313D40A0319D50A1E28861106124C3020
:101070008E210A128A1577088316D0007608CF00D1
:10108000013050022C3003194F02031C79146430D4
:101090008312CF00D00128210A128A1552308E21E6
:1010A0000A128A1577088316D4007608D300013017
:1010B00054022C3003195302031C7915DE308312BD
:1010C000C0009930C100831650088312C3008316F4
:1010D0004F088312C200831654088312C50083167A
:1010E00053088312C400A03057270A128A15A03073
:1010F000CD000130CE0046270A128A158D30CD0072
:101100009A30CE0046270A128A15861400308618B7
:1011100001308316D9008312D401D5016400E83070
:1011200083120313CF000330D00028210A128A153E
:1011300083120313D40A0319D50A0030550207306D
:1011400003195402031C8E287830C0009A30C10065
:10115000831660088312C30083165F088312C200DF
:10116000A03057270A128A15A030CD000130CE00DA
:1011700046270A128A15B0210A128A15D401D50110
:101180006400E83083120313CF000330D00028211D
:101190000A128A1583120313D40A0319D50A0030E0
:1011A00055020A3003195402031CC0289330CD00A5
:1011B0009A30CE0046270A128A158610003086180B
:1011C00001308316D9004C308E210A128A15770817
:1011D0008316D2007608D100003052026530031920
:1011E00051020318F91464308312CF00D001282172
:1011F0000A128A1552308E210A128A157708831630
:10120000D6007608D5000030560265300319550225
:101210000318F915DE308312C0009930C10083161F
:1012200052088312C300831651088312C20083162A
:1012300056088312C500831655088312C400A030D7
:1012400057270A128A15A030CD000130CE00462F54
:1012500072290730D2007D30D100D10B2D29D20B5D
:101260002D2908002130D2007630D100D10B36294B
:10127000D20B3629000008004130D200EE30D100F8
:10128000D10B4029D20B4029000008008230D20047
:10129000DD30D100D10B4A29D20B4A294F29080051
:1012A0000630D3001330D200B130D100D10B562913
:1012B000D20B5629D30B56295D290800B630C00041
:1012C0009930C1005008C3004F08C200A030572712
:1012D0000A128A15A030CD000130CE0046270A122E
:1012E0008A1546295008003A03197A29033A031946
:1012F00088295E294F08053A031929291C3A031940
:1013000032292B3A03193C29563A031946295E29FA
:101310004F08E83A031950295E2908008312031385
:10132000A6000730831603178800031385004C308E
:101330008312260603199E2902309F290130C321FA
:101340007408A8007308A7002808A5002708A400AF
:101350000310A50CA40C2408F6002508F7000800CB
:1013600085163230CF00D00128210A128A15831247
:1013700003138616C830CF00D0012821831203132F
:1013800086128512080083120313A1000F30A105F5
:10139000C3309F052108F50001300310F50DFF3E15
:1013A0000310031DCE29750D9F041F14F930F5009D
:1013B0000000F50BD829DC290000831203139F14C9
:1013C0009F18E0291E08A300A20183161E0883129D
:1013D000A2070318A30A1F102308F4002208F30031
:1013E00008002830CD009830CE004627D401D50122
:1013F000A830A300A40183165F08FF3E8312A50056
:10140000831660080318013EFF3E8312A6000A16E9
:101410008A1140260A128A1555082402031D122A31
:1014200054082302031C432A540854075407D300CA
:101430002F30C0009930C1005508C3005408C200C5
:101440005308123E5C240A128A15643E0313C4003A
:10145000003003180130C5005308133E5C240A1203
:101460008A150313C600C7015308143E5C240A12F0
:101470008A150313C800C90171240A128A15D40AF7
:101480000319D50AF8290C30F400F50150240A128A
:101490008A1575080313D0007408CF000830F400D3
:1014A000F50150240A128A1575080313D200740836
:1014B000D100F030C0009830C1008316600883125C
:1014C000C30083165F088312C20071240A128A15B2
:1014D0006730C0009830F6270A128A1571240A1264
:1014E0008A150E30F400F50150240A128A15750889
:1014F0000313D0007408CF000A30F400F501502423
:101500000A128A1575080313D2007408D1009930A5
:10151000C0009830F6270A128A15712CA830A30053
:10152000A401831660088312A60083165F08831245
:10153000A5000A168A1140260A128A152308E4001B
:101540002408E500640864076407E900123EE4002B
:10155000003003180130E500803AFF0080307F0240
:10156000031DB42AFE30640203180800A830831259
:101570000313AA00AB01831660088312AD00831623
:101580005F088312AC000A168A116A260A128A15AD
:101590002A082B04031D092B0A128A1135240A126A
:1015A0008A155F08E8005E08E7009C30E70703182B
:1015B000E80AFF30E8076808803AFF0081307F02C0
:1015C000031DE42A00306702031CEA2AFF3083125D
:1015D0000313F12A83120313E81FF02AE601F22A0B
:1015E0006708E6006608F4006908123E35240A120E
:1015F0008A15F401831203136908133E35240A1275
:101600008A15F401831203136908143E35240A1263
:101610008A15790803190800791C2B2B3A3083129C
:101620000313CD009A30CE0046270A128A150C30DB
:10163000A100A201F400F50150240A128A157408D1
:10164000013E0313A30075080318013E003EA400E9
:1016500028240A128A15F91C4A2B4C3083120313D2
:10166000CD009A30CE0046270A128A150E30A1000E
:10167000A201F400F50150240A128A157408013EF3
:101680000313A30075080318013E003EA40028249C
:101690000A128A15791D692B433083120313CD007A
:1016A0009A30CE0046270A128A150830A100A201FE
:1016B000F400F50150240A128A157408013E031340
:1016C000A30075080318013E003EA40028240A1256
:1016D0008A15F91D882B543083120313CD009A30DC
:1016E000CE0046270A128A150A30A100A201F40092
:1016F000F50150240A128A157408013E0313A30051
:1017000075080318013E003EA40028240A128A1519
:1017100079188C2BF91C9B2B831203136908133E39
:101720005C240A128A15013EF40003136908133E73
:1017300035240A128A15831203136908143E5C24A7
:101740000A128A15013EF40003136908143E352479
:10175000F90108008312EA006A080319F22BA53088
:10176000CD009A30CE0046278316DF01E0010A162D
:101770008A11C9260A128A150C30A100A201A30100
:10178000A40128240A128A150E3083120313A10023
:10179000A201A301A40128240A128A150830831289
:1017A0000313A100A201A301A40128240A128A158F
:1017B0000A3083120313A100A201A301A40128246B
:1017C0000A128A151230F40135240A128A151330D0
:1017D000F40135240A128A151430F40135240A1252
:1017E0008A15F92B7F30CD009A30CE0046270A1299
:1017F0008A1583160313DA01DA0A5A08F400033053
:1018000035240A128A1508200A128A158E220A1215
:101810008A1583160313DF0A0319E00A10308312B6
:10182000A100A201831660088312A40083165F083A
:101830008312A30028240A168A1154230A128A1537
:10184000053080240A128A15003A031D0800032C73
:101850002408F400210835240A128A158312031380
:101860002308F4002108013E352CF50083160317E8
:101870008C18362C750883128D0074088C003F304C
:1018800083168C0503108B1B03148B130C1555301A
:101890008D00AA308D008C140C1103188B170800D2
:1018A0007408013E5C240A128A15F60074085C2450
:1018B000F5007608F4000800F300640083160317AF
:1018C0008C185D2C730883128D003F3083168C05B5
:1018D0000C1403100C1803140318013083120C08A5
:1018E00008000130CB01CC004230CA004008AE00F5
:1018F0004108AF004A30B0004B300A168A112B2C39
:101900008312D400D630CD009A30CE0046270A127A
:101910008A155408D500550803190034BA30C000A0
:101920009A30C1005508C200C30171240A128A15F9
:10193000DC270A128A15031801346400E830831288
:101940000313CF000330D00028210A128A15831216
:101950000313D5038B2C6C08003A0319DA2ED52E0D
:101960000A168A1154230A128A150A168A111B288C
:101970000A128A112428D030C0009A30C100831680
:101980006E088312C30083166D088312C200A03054
:1019900057270A128A15A030CD000130CE00462FFD
:1019A0000A168A111B280A168A15EC2DD030C000A1
:1019B0009A30C10083164C088312C30083164B086B
:1019C0008312C200A03057270A128A15A030CD001A
:1019D0000130CE00462F0A168A11F32ED030C000F7
:1019E0009A30C100831658088312C3008316570823
:1019F0008312C200A03057270A128A15A030CD00EA
:101A00000130CE00462F8614003086180130831630
:101A1000D900E2308312CD009A30CE00462F8610D6
:101A20000030861801308316D900E0308312CD00D3
:101A30009A30CE00462FCC30C0009A30C1008316B9
:101A400059088312C200A030C30157270A128A1511
:101A5000A030CD000130CE00462F0A168A11152A7B
:101A60000A128A1135240A128A155F088316B400F7
:101A700083125E088316B3000A128A1135240A12F3
:101A80008A155F088316B60083125E088316B500B8
:101A90000A308312A300A401831634088312A6001F
:101AA000831633088312A5000A168A1140260A12EB
:101AB0008A1524088316B800831223088316B700FA
:101AC0000A308312AA00AB01831636088312AD00D8
:101AD000831635088312AC000A168A116A260A1288
:101AE0008A152B088316BA0083122A088316B900B8
:101AF00071308312C0009A30C100831638088312F7
:101B0000C300831637088312C20083163A08831273
:101B1000C500831639088312C400A03057270A1263
:101B20008A15A030CD000130CE00462F7430C000A1
:101B30009A30C1004C308E210A128A157708C300F2
:101B40007608C200A03057270A128A15A030CD00AF
:101B50000130CE00462F7430C0009A30C1005230A0
:101B60008E210A128A157708C3007608C200A030B9
:101B700057270A128A15A030CD000130CE00462F1B
:101B80004C300A168A15AC2D52300A168A15AC2D27
:101B90000616E230CD009A30CE00462F0612E03015
:101BA000CD009A30CE00462F8615E230CD009A3017
:101BB000CE00462F8611E030CD009A30CE00462F61
:101BC0004C300A128A118B2F52300A128A118B2F35
:101BD000B02908280A168A156F2DD130C0009A3016
:101BE000C10000305C240A128A150313C200A03021
:101BF000C30157270A128A15A030CD000130CE004C
:101C0000462FC830CD009A30CE00CF270A128A1551
:101C1000A030CB270A128A156B270A128A152308CF
:101C20008316BF0012308312CD009A30CE00CF272A
:101C30000A128A15A030CB270A128A156B270A12BE
:101C40008A1523088316C00008308312CD009A300D
:101C5000CE00CF270A128A15A030CB270A128A1588
:101C60006B270A128A1523088316C1001C308312C1
:101C7000CD009A30CE00CF270A128A15A030CB278C
:101C80000A128A156B270A128A1523088316C200C6
:101C900026308312CD009A30CE00CF270A128A1543
:101CA000A030CB270A128A156B270A128A1523083F
:101CB0008316C30030308312CD009A30CE00CF2778
:101CC0000A128A15A030CB270A128A156B270A122E
:101CD0008A1523088316C400FE308312CD00993084
:101CE000CE00CF270A128A15831640088312DB0024
:101CF000831641088312DC00831642088312DD003C
:101D0000831643088312DE00831644088312DF0023
:101D1000A030CB270A128A156B272308E000831610
:101D20003F080A128A11DE29F1290A168A11C926EA
:101D30000A128A1576088316BE007508BD0074085D
:101D4000BC007308BB00BB300A168A11AA260A120F
:101D50008A15CD000130CE00462F0130AA2B00306D
:101D6000AA2B8316DA015A08F400033035240A122C
:101D70008A15BF3083120313CD009A30CE00462F50
:101D8000D130C0009A30C100831660088312C300AE
:101D900083165F088312C200A03057270A128A15E3
:101DA000A030CD000130CE00462F6A30CD009A30F1
:101DB000CE00462F6B08013A0319B02C033A0319E1
:101DC000D02C013A0319AD2E073A0319AF2E013A70
:101DD0000319B12E033A0319C02E013A0319B82C86
:101DE0000F3A0319BB2C013A0319D32C033A0319F8
:101DF000D62C013A0319EB2C073A0319EE2C013AC1
:101E000003192D2D033A0319302D013A0319EA2D38
:101E10001F3A0319ED2D013A0319012E033A031954
:101E2000952E013A0319032D073A03190F2D013A94
:101E300003191B2D033A0319962D013A0319AB2DF3
:101E40000F3A0319C02D013A0319C42D033A03199F
:101E5000C82D013A0319CE2D073A0319D42D013AA2
:101E60000319DA2D033A0319E02D013A0319E42D81
:101E70003F3A0319E82D013A0319E82D033A0319F3
:101E8000E92D063A0319942ED52E08008630C0009D
:101E90009A30C100D430C2009A30C3004D08C4004B
:101EA0004E08C500D430C6009A30C700712CC70058
:101EB000C8004230C901C6004008AE004108AF006A
:101EC0004630B00048300A168A112B244808840096
:101ED0008317800108000313AA002A088400203019
:101EE0000006031D752FAA0A6D2F2A0884000930E9
:101EF00000060319732FA801A901A7012A0884006D
:101F00002D300006031D862FA70AB52F2A0884004E
:101F10002B3000060319B52F2A08840000080A1682
:101F20008A1132260A128A15031CB72F2A08840048
:101F30002908F4002808F3000A30F500F6010A1613
:101F40008A118E260A128A15831700087307A500C6
:101F50000030031801307407A6002508D03EA80001
:101F600026080318013EFF3EA900AA0A8C2F270865
:101F70000319C62F2809A5002909A600A50A0319D7
:101F8000A60A2508A3002608A40008002908A40022
:101F90002808A3000800F5000A128A11092F8830CA
:101FA000C0009A30C100D430C2009A30C3004D083E
:101FB000C4004E08C500712C83120313981CED2F2A
:101FC000831698129816831218121816EB2F1A08F7
:101FD000831698129816031008001819E72F7A082C
:101FE00083165B060319EB2F03140800C100500889
:101FF000C3004F08C2005208C5005108C4000800C1
:10200600F8100C18F814831603130C104A08F6007F
:102016004908F500F81C1328831603130C14162818
:10202600831603130C107608F4007508F3000800F5
:10203600063083166F0203182F2803106F0DE13E3A
:102046008400831300088312CD00840A00088403E9
:10205600CE000A128A15462FE4308312CD009A303C
:10206600CE000A128A15462F831203138C1E51289E
:1020760083168C1E51287A08903E840083121A0813
:10208600831780007A08013E8316DC000F30DC05DA
:102096005C085B06031951285C08FA0083120C1EC3
:1020A600662883160C1E66285E08103E8400831779
:1020B6000008831299008316DE0A0F30DE055E08DB
:1020C6005D0603190C1283160C1C7E2883120C1C49
:1020D6007E28101080308F008E0110148316C90AD6
:1020E6000319CA0AC50A0319C60A0319C70A031936
:1020F600C80A83120C1072088A0071088400700ED8
:102106008300FE0E7E0E0900B80084000008B900A8
:10211600840A0008BA00840A0008BB00840A000882
:10212600BC003C308E270A168A117D210A168A11B8
:10213600220883160317DC00831203132108831673
:102146000317DB003C3074270A168A11AC220A16E4
:102156008A11CA270A168A113C308E270A168A1156
:102166007D210A168A11220883160317DE008312C0
:102176000313210883160317DD003C3074270A1663
:102186008A11AC220A168A11CA270A168A11183031
:102196008E270A168A117D210A168A1122088316AD
:1021A6000317E00083120313210883160317DF00C9
:1021B600183074270A168A11AC222A0883160317C8
:1021C600E20083120313290883160317E10062084D
:1021D600F6006108F5000430F5070318F60A073023
:1021E600F300F4010A168A1573270A168A11740871
:1021F60083160317E8007308E7004630E500E6019A
:10220600BF270A168A11E6210A168A11E5270A1639
:102216008A112F08803A3702031D15292E088316C6
:1022260003176102031C2F2983160317BF270A16FB
:102236008A11E6210A168A112E0883160317E1026F
:10224600831203132F0883160317031CE203E2020B
:10225600E50A0319E60A032983160317660883129B
:102266000313AF0083160317650883120313AE002A
:10227600E6212E08B9000230B90583160317620855
:10228600EA006108E900E301E40183160317630825
:10229600123E840098300318013E83120313FF0098
:1022A6000A168A1500200A168A113904BA00E5278B
:1022B6000A168A1180303702031D65293A088316EB
:1022C60003176102031C7729831203133A08831646
:1022D6000317E102031CE203E30A0319E40A83126B
:1022E60003130310B90C482983160317E10A0319CF
:1022F600E20ADB34F401A81F8D29A509A609A7095E
:10230600A809A50A0319A60A0319A70A0319A80A00
:10231600F401F40AA41F9A29A109A209A309A40990
:10232600A10A0319A20A0319A30A0319A40A240875
:102336002304220421040319CF29F301F30AA41B61
:10234600AA290310A10DA20DA30DA40DA1292408ED
:102356002802031DB82923082702031DB8292208CD
:102366002602031DB82921082502031CC9292108B4
:10237600A5022208031C220FA6022308031C230F12
:10238600A7022408031C240FA8020310A40CA30C04
:10239600A20CA10CF30BAA2974080319DD29A509BF
:1023A600A609A709A809A50A0319A60A0319A70ACF
:1023B6000319A80A2808A4002708A3002608A200D3
:1023C6002508A10008002E080339031D0B2A6430D6
:1023D600AA00AB012F08AD002E08AC006A260A162B
:1023E6008A112A082B04031D102A9030AA000130F6
:1023F600AB002E082C3EAC002F080318013E013E10
:10240600AD006A260A168A112A082B040319102A17
:102416006D30AE000130AF0008006E30AE00013006
:10242600AF0008001130CD009930CE000A128A158F
:10243600CF270A168A11A0300A128A15CB270A1648
:102446008A11A0300A128A156B270A168A112408E7
:10245600D7002308D60000305702C83003195602A9
:10246600031CA52A013057024130031956020318EE
:10247600A52A0130831603178800031385008312EB
:1024860006156430CF00D0010A128A1528210A16D3
:102496008A1100300A128A15C3210A168A11740895
:1024A600D5007308D4000611A9005508AA00AB018F
:1024B600AC015608A1005708A2000330A301A401ED
:1024C600A801A701A600E830A50021230A168A1153
:1024D6002408B0002308AF002208AE002108AD0092
:1024E600AC222A088316CE00831229088316CD0053
:1024F6008312A101A10AA20183164E088312A40029
:1025060083164D088312A3000A128A1528240A1678
:102516008A11D03083120313C0009A30C10083168B
:102526004E088312C30083164D088312C200A030E2
:102536000A128A155727A030CD000130CE000A12A4
:102546008A15462F6A30CD009A30CE000A128A15B7
:10255600462FB201AC1FBC2AA909AA09AB09AC09CE
:10256600A90A0319AA0A0319AB0A0319AC0AB2018C
:10257600B20AB01FCB2AAD09AE09AF09B009AD0A40
:102586000319AE0A0319AF0A0319B00A0130B206DD
:10259600B301B401B501B6012C082B042A042904A1
:1025A60003190A2BB101B10AAC1BDF2A0310A90DCE
:1025B600AA0DAB0DAC0DD62A0310B30DB40DB50D97
:1025C600B60D2C083002031DF22A2B082F02031D1C
:1025D600F22A2A082E02031DF22A29082D02031CBC
:1025E600042B2908AD022A08031C2A0FAE022B0869
:1025F600031C2B0FAF022C08031C2C0FB002331444
:102606000310AC0CAB0CAA0CA90CB10BDF2A3208D8
:102616000319182BB309B409B509B609B30A031986
:10262600B40A0319B50A0319B60A3608AC00350808
:10263600AB003408AA003308A9000800F301F4012E
:10264600F501F601211C3B2B2508F307260803118B
:102656000318013E031DF407270803110318013E62
:10266600031DF507280803110318013E031DF6078D
:102676000310A50DA60DA70DA80D0310A40CA30C01
:10268600A20CA10C2408230422042104031D252BDB
:102696007608A4007508A3007408A2007308A100B8
:1026A6000800C9260A168A11DC270A168A11D327BA
:1026B6000A168A118E267308D4007408D500D6012E
:1026C600D7015408D807550803110318013E031D06
:1026D600D907560803110318013E031DDA075708E8
:1026E60003110318013E031DDB07C530C0009930F6
:1026F600C10083166E088312C30083166D08831209
:10270600C200A0300A128A1557270A168A11A0306D
:10271600CD000130CE000A128A1546270A168A1104
:10272600DC01DD0183164C0883125D02031D9F2B1D
:1027360083164B0883125C020318B32B6400E8303F
:1027460083120313CF000330D0000A128A15282102
:102756000A168A1183120313DC0A0319DD0A952B64
:102766008316981CB32B8C1283129813850186014D
:10277600043087008316D9018312101080308F0031
:102786008E01101483160C140B178B13DD2B031EEE
:10279600FB2B630083120313101080308F008E0111
:1027A60010140C108316C50A0319C60A0319C70AA2
:1027B6000319C80A83125D08D5005C08D400DC0A38
:1027C6000319DD0AD3270A168A118E260A168A11DC
:1027D6007308FF3ED60074080318013EFF3ED7007B
:1027E60055085702031DF92B540856020318CA2B25
:1027F60050270A168A118B17831D031E042C0230DC
:10280600082C831D031A092C0330EF006430831251
:10281600CF00D0010A128A1528210A168A11B0267D
:10282600DD308312CD009A30CE000A128A15462773
:102836000A168A11C9260A168A11DC270A168A116F
:102846005830AA26CD000130CE000A128A15462F2E
:10285600BF0083120313A7270A168A1500200A163B
:102866008A11BE003E0803192F2E25303E06031995
:102876004D2C3F0A8400831300080319492CF427C2
:102886000A128A1100270A168A112C2C9B270A166F
:102896008A112C2CBC01BD01B5012F08FF002E08A2
:1028A60084000A168A1500200A168A1132260A168C
:1028B6008A11031C352DBC01BD010A30F300F40159
:1028C6003D08F6003C08F5008E267408BD00730826
:1028D600BC002F08FF002E0884000A168A15002067
:1028E6000A168A11D03EB100FF3003180030B2003C
:1028F6003108BC070318BD0A3208BD07AE0A031922
:10290600AF0A2F08FF002E0884000A168A15002039
:102916000A168A1132260A168A11031C352D602CD6
:1029260083270A168A11BA00840A00088403BB00AA
:102936003A04031DA22C5C30BA009A30BB00B801E1
:10294600B90138083A0784003B0803183B0AFF0020
:102956000A168A1500200A168A11003A0319B72C9E
:10296600B80A0319B90AA42C3D083902031DBD2C67
:102976003C0838020318C62C3808BC023908031C68
:10298600BD03BD02C82CBC01BD01FF308312031379
:10299600BC07031CBD033C0FD32C3D0A03191C2D99
:1029A6003F0A8400831300080319E02CFA270A1251
:1029B6008A1100270A168A11C82CB3270A168A110B
:1029C600C82C3F0A8400831300080319032D3B0813
:1029D600FF003A0884000A168A1500200A168A1192
:1029E600F3003F0A8400831300080A128A110027A5
:1029F6000A168A1183120313BA0A0319BB0A1C2D7D
:102A06003B08FF003A0884000A168A1500200A16B9
:102A16008A11B1003F08840083130008840031083E
:102A260083178000BA0A0319BB0A3F088400831380
:102A3600800A0130B8020030031CB903B902380F0E
:102A4600E42C390A03192C2CE42C83270A168A1144
:102A5600BE003E30BA00BB01B801B80AB901B72CB6
:102A660035174F2DA7270A168A1500200A168A1130
:102A7600BE00003A03192F2E633A0319282D073A90
:102A860003194F2D0D3A03194F2D1A3A0319932C9A
:102A9600063A0319332D2C2D351B622D83270A1672
:102AA6008A11B600840A0008B700B71F692D0330E3
:102AB600B504B609B709B60A0319B70A692D8327FB
:102AC6000A168A11B600840A0008B700BE0105304E
:102AD600BE0A3E060319852D03103E0DED270A1684
:102AE6008A1500200A168A11B1000A168A150020D6
:102AF6000A168A11B2003702031D832D31083602E9
:102B060003186A2D3C083D040319912D3508033935
:102B16000319912DFF30BC07031CBD033E08B1000D
:102B2600B201B11BB2033208803AB3003D08803AC5
:102B36003302031DA02D3C0831020318AF2D83126A
:102B460003133E08B100B201B11BB203BC02320846
:102B5600031CBD03BD02B32D83120313BC01BD01CB
:102B66003C083D040319D12D3F0A84008313000855
:102B76000319C42DFA270A128A1100270A168A1188
:102B8600C72DB3270A168A11FF3083120313BC0719
:102B9600031CBD033C083D04031DB72D350803394E
:102BA6000319F12D3F0A8400831300080319E62D4B
:102BB6002D30F3003F0A840000080A128A1100270C
:102BC6000A168A11F12D3F088400000884002D3072
:102BD600831780003F0884008313800A831203133F
:102BE6003E08B400292E0A30AA00AB010310340DAA
:102BF600ED270A168A1500200A168A11A3000A165E
:102C06008A1500200A168A11A4003708A60036087D
:102C1600A50040260A168A112408AD002308AC0038
:102C26006A260A168A112A08303EBE003F0A840028
:102C3600831300080319262EF4270A128A11002787
:102C46000A168A11292E9B270A168A118312031344
:102C5600B403340FF62D2C2CAE01AF010800F4009E
:102C66003A30F301740203183E2E30307402031C0E
:102C76003E2EF301F30A730C0800A801A9012308EC
:102C860024040319652EA701A70AA41B4E2E0310C0
:102C9600A30DA40D472E0310A80DA90D2408260286
:102CA600031D572E23082502031C612E2308A502A7
:102CB6002408031CA603A60228140310A40CA30CC4
:102CC600A70B4E2E2908A4002808A30008002A08EE
:102CD6002B040319892EF701F70AAB1B762E031076
:102CE600AA0DAB0D6F2E2B082D02031D7C2E2A0874
:102CF6002C02031C852E2A08AC022B08031CAD03EC
:102D0600AD020310AB0CAA0CF70B762E2D08AB0008
:102D16002C08AA0008008312A101A201731C9A2E96
:102D260075088312A1070318A20A7608A2070310E2
:102D3600F50DF60D0310F40CF30C73087404031D63
:102D4600912E83122208F4002108F3000800831252
:102D5600C20064270A168A15322E19308316031309
:102D660099001815181283129817181698128316B8
:102D76000C128C16181383121813831698129816B1
:102D86000B17DE01DD01DB01FA010800781183165D
:102D960003130C187815831603130C1048088312B6
:102DA600A400831647088312A300831646088312DD
:102DB600A200831645088312A100781DE62E83160D
:102DC60003130C14E92E831603130C108312240824
:102DD600F6002308F5002208F4002108F300080095
:102DE6004A30CD009930CE000A128A15CF270A162E
:102DF6008A11A0300A128A15CB270A168A11A0302A
:102E06000A128A156B270A168A112408D00023088D
:102E1600CF0004305002453003194F020318492FE2
:102E260050088316D80083124F088316D700063041
:102E36008312A100A201831658088312A4008316E8
:102E460057088312A3000A128A1528240A168A1123
:102E5600CC3083120313C0009A30C1008316580881
:102E66008312C300831657088312C200A0300A12C9
:102E76008A1557270A168A11A030CD000130CE00D8
:102E86000A128A1546270A168A11502F6A30CD0073
:102E96009A30CE000A128A15462F7810831603132D
:102EA6000C187814831603130C10C901CA01781C78
:102EB600602F831603130C140800831603130C10DB
:102EC6000800C100840083130008BD00840A0008BE
:102ED600BE00840A0008BF00840A0008C0003D3016
:102EE600872883120313A900AA01AB01AC013C0891
:102EF600B0003B08AF003A08AE003908AD00080044
:102F06003008840083130008B100023080073108BE
:102F1600840000080800A100A201A301A4013C0846
:102F2600A8003B08A7003A08A6003908A500080033
:102F36003F088400000884003E08831780003F088D
:102F460084008313800A08002F08B2002E08B100FF
:102F5600AE0A0319AF0A3208FF00310884000800E0
:102F66003F088400000884002030831780003F0853
:102F760084008313800A0800660883120313AF00D7
:102F860083160317650883120313AE0008002C0886
:102F9600BC002B08BB002A08BA002908B9000800A3
:102FA60083166E08F4006D08F3003C30F500F60158
:102FB60008007608DB007508DA007408D900730883
:102FC600D8000800831603176208803A8312031399
:102FD600B70008001E3E840098300318013EFF002B
:102FE60008003E08F3003F0A84000008080020306D
:102FF600F3003F0A840000080800FF1B0A28831319
:103006007F1883170008840A0319FF0A08007F083F
:103016007F398A000408840A0319FF0A82001F34D4
:103026001C341F341E341F341E341F341F341E3408
:103036001F341E341F34013400340A34003464341F
:103046000034E83403341034273457346534653497
:103056006B3420344E346F342E342C3420345634B2
:103066006F346C34743461346734653420342834F6
:10307600563429342C3420344C3465346634743454
:1030860020345334743472346F34623465342034EB
:103096004634613475346C34743473342C342034CF
:1030A6005234693467346834743420345334743495
:1030B60072346F3462346534203446346134753486
:1030C6006C347434733400340D3420344C34653429
:1030D60066347434203455346E3464346534723452
:1030E6002D344334683461347234673465343A3489
:1030F6002034253433346434093452346934673423
:1031060068347434203455346E346434653472341F
:103116002D344334683461347234673465343A3458
:1031260020342534333464340A3400340D342034E6
:103136004C34653466347434203420344F34763459
:10314600653472342D3463346834613472346734D0
:1031560065343A34203425343334643409345234F3
:103166006934673468347434203420344F34763408
:10317600653472342D3443346834613472346734C0
:1031860065343A3420342534333464340A34003414
:103196004A3461346E344634653462344D346134B5
:1031A60072344134703472344D34613479344A3473
:1031B60075346E344A3475346C344134753467343E
:1031C6005334653470344F34633474344E346F344E
:1031D600763444346534633400340A340D3454345C
:1031E6004F34543441344C3420344634413455340D
:1031F6004C345434533420344F34553454342034FE
:103206004F344634203425346434203449344D3424
:1032160041344734453453340A3400344434653435
:103226006334693476346F346C34743473342834CC
:103236003234303430342D343334323430342C3468
:1032460030343D343D34613462346F347234743416
:1032560029343A34203400340D34203420342034D8
:103266002534323464342C34093409342534333467
:1032760064342C34093409342534333464342C341E
:10328600093409342534333464340A34003431348F
:103296002D34313430343934323420346D34693499
:1032A6006E342C3430343D343D3466346F347234ED
:1032B600653476346534723429343A342034003433
:1032C600573461346B34653479342034253473349F
:1032D6002034433461346D346534723461342034BF
:1032E60054347234693470346F34643421340034A5
:1032F600533475346E344D346F346E3454347534FF
:10330600653457346534643454346834753446341B
:103316007234693453346134743400344134633460
:103326007434693476346534203444346534703406
:103336006C346F3479346D3465346E3474342134BE
:10334600003431342D343234353435342C34303481
:10335600203474346F342034613462346F34723400
:1033660074343A3400344E346F3420346434653463
:103376006C346134793420342534643420346D342B
:103386007334003453346C3465346534703420340B
:103396002534643420346D3469346E340034313469
:1033A6002D34313430343934323420346D34693488
:1033B6006E343A3400344C343A3425347534563449
:1033C600203452343A342534753456340034433478
:1033D600683461347234673465342E342E342E34B6
:1033E600003430342D34363430342034733465347C
:1033F60063343A3400344434533454342834303447
:103406002D34313429343E340034443444342834A1
:1034160031342D343334313429343E3400344D3490
:103426004D34283431342D343134323429343E3459
:10343600003448344834283430342D34323433346C
:1034460029343E3400344D344D34283430342D3450
:103456003534393429343E34003453345334283423
:1034660030342D343534393429343E3400344C3438
:103476005334203475346E34643465347234003415
:1034860052345334203475346E34643465347234B3
:1034960000344C34533420346F347634653472340B
:1034A60000345234533420346F34763465347234F5
:1034B600003428346E3475346C346C34293400345A
:1034C6002534633420342E342E342E3400347634AE
:1034D60031342E3434342E343234003425347534B9
:1034E6002E34253475345634003449346D346734FB
:1034F60020342534643400345234653473347534DE
:103506006D346534003425347334253473342534EE
:1035160073340034433461346D3473342B340034E3
:10352600433461346D3473342D340034523453349F
:1035360054345734443400345234533454344F34AE
:103546004B34003442346534673469346E340034A5
:103556002534633420342134003457344B34573403
:103566004434003457344B344F344B3400340D3428
:103576002534333464340034483461346C34743460
:10358600003454344F3421340034593459343E34E1
:1035960000343D342534643400343D3425347534E8
:1035A60000340D340A3400343E34203400345434AC
:1035B6004F340034553470340034303400343134F0
:0635C60000343F34003424
:103ADE00A430CD009930CE000A128A15CF270A16CF
:103AEE008A15A0300A128A15CB270A168A15A0301D
:103AFE000A128A156B270A168A152308CF004F085B
:103B0E000319A52D4F08F40000300A128A1535242A
:103B1E000A168A15D03083120313C0009A30C100E2
:103B2E004F08C200A030C3010A128A155727A030D1
:103B3E00CD000130CE000A128A15462F6A30CD0014
:103B4E009A30CE000A128A15462FD6004C3A031D23
:103B5E00B22D0616B32D86156330C0009A30C10003
:103B6E005608C200A030C3010A128A1557270A163A
:103B7E008A15A030CD000130CE000A128A154627D4
:103B8E000A168A15D401D501003055021E300319CC
:103B9E0054020318E42D6400E83083120313CF009F
:103BAE000330D0000A128A1528210A168A158312AC
:103BBE000313D40A0319D50ACB2D4C305606031D18
:103BCE00EA2D0612080086110800F430CD00993057
:103BDE00CE000A128A15CF270A168A15A0300A12AD
:103BEE008A15CB270A168A15A0300A128A156B275A
:103BFE000A168A152408D0002308CF000030500280
:103C0E003D3003194F0203182B2E50088316CC009B
:103C1E0083124F088316CB00CC308312C0009A302B
:103C2E00C10083164C088312C30083164B088312FF
:103C3E00C200A0300A128A155727A030CD000130DD
:103C4E00CE000A128A15462F6A30CD009A30CE0069
:103C5E000A128A15462F83120313AC007B30AA007A
:103C6E009930AB000330F3002C080C3E8400831710
:103C7E0000082027AA070318AB0AA900A91BAB034B
:103C8E00C03083120313AD002B08FF002A088400F6
:103C9E000A168A1500200A168A15E9270A168A15A9
:103CAE0000200A168A15E9270A168A1500200A1618
:103CBE008A15A9002D088400290883178000AD0AF3
:103CCE002D08840020308000CB30AD0AAA00983039
:103CDE00AB000330F3002C08083E840000082027B8
:103CEE00AA070318AB0AA900A91BAB03831203137F
:103CFE002B08FF002A0884000A168A1500200A16CF
:103D0E008A15E9270A168A1500200A168A15E92748
:103D1E000A168A1500200A168A15A9002D08840095
:103D2E00290883178000203083160317C7008312DB
:103D3E0003132C08063E84000008A5002030A600C0
:103D4E00A700CA30F9260A168A152C08043EF82751
:103D5E000A168A15CD30F9260A168A152C08023E47
:103D6E00F8270A168A15D030F9260A168A152C0855
:103D7E0084000008A5003030A6002030A700D33004
:103D8E00F9260A168A156430F300F4012C080A3E4F
:103D9E0084000008F500840A0008F6002E270A1693
:103DAE008A157308133EA5002030A600D630A70151
:103DBE00F9260A168A156430F300F4012C080A3E1F
:103DCE0084000008F500840A0008F60073270A161E
:103DDE008A157308A5003030A6000A30A700D83027
:103DEE00F926C034A8008400270883178000A80392
:103DFE00280884000A30F3002508CD270A168A15F4
:103E0E00303E80000A30F3002508B2270A168A15C4
:103E1E00A500250803191A2FA803280884002508D1
:103E2E00303E80000800A803280884002608800081
:103E3E000800F500F40173087518F4070310F30D6C
:103E4E000310F50C7508031D222F74080800A2013B
:103E5E00F41F382FF309F409F30A0319F40AA20127
:103E6E00A20AF61F412FF509F609F50A0319F60AFB
:103E7E000130A206A301A401730874040319662F6E
:103E8E00A101A10AF41B4F2F0310F30DF40D482FBF
:103E9E000310A30DA40D74087602031D582F73088A
:103EAE007502031C622F7308F5027408031CF603D7
:103EBE00F60223140310F40CF30CA10B4F2F22085F
:103ECE0003196E2FA309A409A30A0319A40A24082F
:103EDE00F4002308F300080083120313A201F61F57
:103EEE007F2FF509F609F50A0319F60AA201A20AAF
:103EFE00F41F862FF309F409F30A0319F40A730861
:103F0E0074040319A52FA101A10AF41B922F03100B
:103F1E00F30DF40D8B2F74087602031D982F730882
:103F2E007502031CA12F7308F5027408031CF60317
:103F3E00F6020310F40CF30CA10B922F22080319B6
:103F4E00AD2FF509F609F50A0319F60A7608F400FD
:103F5E007508F3000800F400F60173080319CB2F5F
:103F6E00F501F50AF31BBE2F0310F30DB82F031046
:103F7E00F60D73087402031CC82F7308F40276142E
:103F8E000310F30CF50BBE2F76080800F500083071
:103F9E00F600F7017508F40007300310F40CFF3E2D
:103FAE000310031DD52F770D7404F7000310F50DC4
:103FBE0073087702031CE52F7308F702F60BD12F57
:103FCE0077080800A9002D088400290883178000AF
:103FDE00AA0A0319AB0AAD0A2B08FF002A088400AF
:103FEE00080084000008A5003030A6003A30A70073
:023FFE000800B9
:02400E00DAECEA
:00000001FF
